:020000040000FA
:10000000850186018316EF2AFF00FF0E030E830190
:10001000D3000408D4008C10BE0B11283230BE006F
:10002000BD17C7082B1C0319172886161828861217
:10003000AA0F2A28A90F2A28AB0A7D153C30AA004E
:10004000F630A9002B182A28C708031DC70B2A2839
:1000500006128612CB186F28CB1D3428CC0B6F28C4
:100060000519CB11CC0A6F284B1C3E2805196F28A7
:100070004B10CD010430CE0006305F2805084B063A
:10008000043903194928CB064B1602304B1B0630A6
:10009000CC004B1B5628CC0B6F28031005190314FA
:1000A000CE0DCD0D4B174B1204305F284B1A612833
:1000B000CC0B6F284B0882390938CB008030CC003C
:1000C0006F284B13CD1F6F28CE0DCD0D4E0DCD0DCE
:1000D000CE134D1FCE17CD1A0314CE0CCB14851E94
:1000E000C303851AC30AC20BEF286430C200C00ADA
:1000F0000319ED280301C31B2030C301C3174106B8
:1001000020390319EF28C106411C9628C11A9D28E1
:10011000B5304007031C8F28E73E031C912841118E
:10012000EF28E430C105BF01BF039828C11A9F28FA
:10013000E2304007031CED28BF0AC001EF28F13070
:1001400040070318ED28F9304007031CA928C11700
:10015000AE28FD304007031CED28C113C00141113A
:10016000C63084003A303F020319DF28083E0318E6
:10017000D92880018403083E0318D928800184030C
:10018000063E0318D92880018403013E0318DF28A6
:10019000063E0318D92880018403013E0318DF2896
:1001A000073E0318D9288001013E0318C11BEF2820
:1001B000ED28410D800C0830C11BC106EF28083026
:1001C000C11BC106C119EC283A303F060319C118FA
:1001D000EF28C40A4115EE284116C11441145408F1
:1001E0008400530E83007F0E0900AB013C30AA004F
:1001F000F630A9000800F101F10AF63E0318FC28C8
:100200000A3EF103F10E710708005F261C21031D51
:100210000D294808C70006161721F10B06291C21D5
:10022000031D080063080319013EE2005715AB24C3
:100230007D142125FD1408002D080006F000840A15
:100240002C080006840A70040800FD101F3071217C
:10025000FD1B2B1C482186102530840007308A00A6
:1002600000081F39CC27801B40387D1C0030FB0064
:1002700008300611FB1F8611FB1B8615FB0D0615AA
:10028000FF3E031D39298403841A2E298614080091
:100290002B1C4C29571970297C1A1C2A8A007C08AF
:1002A0000F398207002AF329EA29C7299C29AE2998
:1002B000B62986297D297829182AC129D729D7293D
:1002C000D72951080F39A100510E0139A00018306B
:1002D000A2001E30A30052080F39A500520E152AA5
:1002E0000830A000A100A200A300A400A5000134D2
:1002F0001830A200A3006108CF2957080339E5216F
:100300000A30A2001A30A3005508CF29FE1B9329FA
:100310007E0828073F39E5210030A71B323E271B06
:10032000193EED2197291B30A000A100A200A117C2
:100330001D30A4000C3076290D30A0000C307D1F3C
:100340001E30A1004508CF214408D321A300A921D4
:10035000F129700E0F3903191F3008004908E521F3
:100360001130A2000530A3004A08CF291A303D18E9
:100370000D30A0000530A2000E30A3007D0E033921
:10038000CF291830A2000D30A3006308CF290D300B
:10039000A2000A30A300330AE521FD190C30D32155
:1003A000A500A921162AFB20F0000F3908004C3EB9
:1003B0008400000E0F39CF210B30A200041C103036
:1003C00084181830A300570E0739D321A100A921A2
:1003D000A00018343108FA213008D321A300700E90
:1003E0000F39A20008002F08ED212E081222300834
:1003F000FA210F2AD321A100700E0F39A0000800A6
:100400002D08FD19B624E5212C08ED212F221222FA
:100410002B1C080044084507E23E0318A517A11746
:10042000A3170800D321A500700E0F39A4000800FF
:10043000C030840018301F2AA5247C080F39A10081
:100440000A30A0001830000603192C2A0008A52144
:10045000A317840A0008122AA3010F30752903107C
:100460002B0C08009E25CB174D08D10050061F39D4
:10047000D01B0039031DE82A4E08D200CF0603190D
:10048000E82A7F39F0004030F100F11AE82A7108BB
:100490004A27F10A7006031D452AFD1402308A001E
:1004A00071031F398207862A812A892A8E2A982A6F
:1004B0009F2AA72AB02AB82AC12AC92AE22AD12A01
:1004C000E02ADD2A732A772A752A522C772C0D2DE3
:1004D0000D2D0D2D0D2D0D2D0D2D4F2DF32CD22C61
:1004E000C92CD02CCB2CC701E82A4925E82A79222F
:1004F000E82A7C0A183A031D183A7C061F39FC06C4
:100500001A29AB0AAB0A78302B020318AB01F6208C
:10051000E62AAB027830031CAB07872A9022E62A32
:10052000AC0A3C302C060319AC0008003D1C902A94
:100530009A22E62AAC03AC1FE62A3B30942AA12279
:10054000E62AAD0A18302D060319AD000800AB22CB
:10055000E62A3D1CA12AAD03AD1F08001730A52ACD
:10056000B222E62A32032E060319AE01AE0A0800B3
:10057000BC22E62A3D1CB22AAE0B08003203AE00B4
:100580000800C322E62A0C302F060319AF00AF0A79
:100590000800CD22E62A3D1CC32AAF0B08000B3011
:1005A000C62AD322E62AB0036330B01F0800B00089
:1005B000B1036330B11BB1000800D8220230E42A35
:1005C000B10ADE2AB00A0130FC00E72AFC01042649
:1005D0004E08CF00CB10CB1F0800F0241729C030E5
:1005E00086008112F93092008C14831207309F002C
:1005F000203084008001840A841FFA2AC603C317AE
:100600006430C20041143E304A273F390319013E8D
:10061000C8003F304A27D0004B1460304A270739C2
:10062000483EE400E4076408F8000130F900203097
:100630000C275725ED260C275C25ED260C27462593
:100640000130F726A038E500AB251026172105302C
:1006500092008C01C0308B00CB1832224108173930
:10066000043A0319DD257D1D792BFD14A926502799
:10067000B300640AF800F901F826A70046252B18F4
:10068000462BA608031DA60B462BFC017425FC086F
:10069000031D532B2B067D1B031D532BF024013010
:1006A0002C1C0730FC00AB08031D792BD608031D5A
:1006B000D60B5C2B57184B25E20857190319632BEF
:1006C000E20B632B571146082C060319692BC6064B
:1006D00005212C08031D792B4408C500C4019C2466
:1006E000C7080318031D792B0130FD1AB6247D1AA3
:1006F000C7002C03FB001E302B067B04031D8B2B35
:10070000B2242D08F300610803198B2BF500A627EE
:100710007608031D0826FD182521BD1F322CBD13A8
:100720000310051E0314B40D34090319A32BC03A9A
:1007300032300319B8003408FE3A031DAA2B3C1EC0
:10074000A72B3C12AA2BB80BAA2B3C16FC173C1467
:100750003230B8000310851D0314B50D3509031997
:10076000BD2BC03A32300319B9003508FE3A031DDB
:10077000C42BBC1EC12BBC12C42BB90BC42BBC1682
:10078000FC17BC143230B9003C0830390319FC1393
:100790003C1CFB2B3C10ED243C1AD02B4925322C61
:1007A0007D1CCE2BAB24A5247C1A2F2C0330AE2429
:1007B0008207A922312CCB22312C7025312CFD113E
:1007C000352C7D13352CC90A012D1030332CA80A85
:1007D000BF2CE024322CF524322CF823322C5E2559
:1007E000322C5225322C5225322C5225322C322CCE
:1007F000C03084002F2CBC1C322CBC10ED24BC1A41
:10080000072C7D1C052C7922322C4925322C7D1C8D
:10081000052CAB24A3247C1A2F2C0430AE24820791
:100820009622312CBA22312C6C25312CFD15352C19
:100830007D17352CCA0A012D0A25322CA803BF2C9E
:10084000DE24322CF724322C4024322C6825322C22
:100850001225322C1225322C1225322C322C422415
:10086000322C04262C2B3724322C3B24322C7D07AF
:100870007D063039FD061430F9007D0878390C2FDB
:10088000C1308400800A041004087F39F90019304F
:100890004A243C30801B80070002031880000008B7
:1008A000840A0C2FA5247C1AD52C0430AE24820790
:1008B000A922C52CCB22C52C7025C52CFD11D82C06
:1008C0007D13D82CC90ADA2C1030DC2CA80ABD2CD8
:1008D000E024E82AF524E82AF823E82A5E25E82A15
:1008E0005225E82A5225E82A5225E82AE82AA32494
:1008F0007C1AD52C0430AE2482079622C52CBA224D
:10090000C52C6C25C52CFD15D82C7D17D82CCA0AF2
:10091000DA2C0A25E82AA803BD2CDE24E82AF724CD
:10092000E82A4024E82A6825E82A1225E82A122520
:10093000E82A1225E82AE82A49082D02031C0800A3
:100940002D0A4A0208000314A62C03107C0D0F394F
:10095000A03E840008005508D60008008A007C0DDF
:100960001E390800F001F101F20108002D08F43EE3
:10097000031C2D0803190C3E0800C124E82AC124D9
:10098000322C1730F90028080C2FFD137D15CB16DB
:10099000E82AA524CC2CA3247C1EE82A8003D62C8C
:1009A000A324D32CA5247C1EE82A800A4324E82A09
:1009B0003B24E82A0325E82A3724E82AD50AE52C2F
:1009C0000130570757060339D7061930F900570881
:1009D0000C275530840064304A2CAB24C701FD1429
:1009E0000A30A60008001030E42AE103F82CE10ADE
:1009F0001930F90057080C271B30F90061308400CA
:100A0000082D0325322C1530F900493084000825C3
:100A100018304A2C0130BD0608009C3E13250408FE
:100A2000B43EE42A993E8400840C1030031CF0305C
:100A300080071D30F90058080C2759080C275A0860
:100A40000C275A08F400590E58047D183B2DF40168
:100A50002F22FB20F10EF10A0F390030D718031DA9
:100A60003B2D1030571F3B2D7119F4041130F11C30
:100A7000F039711C0F39F300552573080C27740EDB
:100A80000C275A2573080C27740E0C27D030F80059
:100A90003C347D1C1729D6017D10CB13212D522506
:100AA0000C30E42A1030D707F82C1430F90040300D
:100AB000F80000341430F9004230582D63083B3AF6
:100AC000031D3B3A013EE3001C30F90063080C2F84
:100AD000630B6B2D3B30632D3D18D32AB00F0800FC
:100AE0003D18D82AB10A0800571E212D2F2203399C
:100AF0000319571E8B2DD71A842D9925DE079925AA
:100B0000DF079925E0078B2DB325DE00700EF03945
:100B1000DF009025E000600EF4005F0E5E04252DDE
:100B20000F30F0057015B325F00B932DF000F03960
:100B30000800A025650E6506103908000108E506C5
:100B40000310E50D650EE039E50C650765076507DF
:100B5000353CE5000800A025E600650EE700A0256D
:100B6000E900650EE8006608EB00EC00EA006708A3
:100B7000ED00EE00ED0DEB0DED0D6B0DEA06EC0C4E
:100B8000EE0C6E08EA06EC0C6E0CEA066708E6004E
:100B90006808E7006908E8006A08E90008008403BB
:100BA000000CF000700C3F39F3000F39731A0A3E45
:100BB000F31A143E731B283E0800C6308400000858
:100BC000D4253006F100B0068403000CF000F00CD0
:100BD000700C1F39D4252F06F104AF06CF252E0641
:100BE000F104AE06CF252D06F104AD068403000CFA
:100BF0007F39D4252C06F104AC062F22F1044111D3
:100C0000F520F108031908007D15CB16FD13080027
:100C10001030F726F600F826FF3A7606031D080086
:100C20000030F726D425AB00AB07F620F826D425F4
:100C3000AC00F826D325AD00F826F826D325AE0063
:100C4000F826D425AF00F826D425F2001030F72678
:100C5000B000F826FF3A3006031D662E1230F72644
:100C6000B100F826F8267D067839FD06F826C90079
:100C7000F826CA00F826A800F826F8265706FB39F9
:100C8000D706F826D500F826E100F826E300F82676
:100C9000D800F826D900F826DA005F26F10AF826EF
:100CA0008000840AF8268000840AF10B4F2E300859
:100CB0007206033903190800B00AA926E52E203070
:100CC000F900A03084000830F10008000C30AD00BD
:100CD000AC01AB010130AE00B301AF00B000143085
:100CE000B1008030EE260230F9002D080B27ED26EA
:100CF0001330F9000030FC000C27FD170C270830DA
:100D0000C9000C271430CA000C270030A8000C279B
:100D10000C270330D7000C275A30D5000C2706309B
:100D2000E1000C271E30E3000C277030D8000C27A0
:100D3000D9000C27DA000C275F26F10A1830800052
:100D40000C27840A003080000C27840AF10B9E2EA9
:100D500008002B3084007830F0263C30F026183024
:100D6000F0262030B2002F08F000AF19F00A701CF6
:100D7000B203023A031DC32EB2033008031931082F
:100D80000339031DB2033208F0260318AE0A0D30F2
:100D9000F0260318AF0AF02631020318B1017D11C5
:100DA000CB1E0800F9012F2280380B272C080B27B7
:100DB0002D080B2733080B272E080B272F080B278E
:100DC00030080B272F220B27CB121030F9003008E8
:100DD0000C2730090C2731080C2F0030F9010C2F9B
:100DE000000203188000840A0318800A6434F900A2
:100DF00017272A272927172701382A27781C042F85
:100E00001C277A08FE0035271C2737271327F90AE5
:100E10007A0883120800FB20FA0017272A272927BF
:100E20007A082A27062F392742278514432F83164D
:100E3000152742273927402F1527F31542278312FC
:100E40000310851803148316FA0D4027F30B1E2F89
:100E500008007908FB000830F300FB1B1527FB1F77
:100E600039273B27FB0DF30B2D2F3927382F15275B
:100E70003B278510432F05140830FF3E031D3D2FEF
:100E80000510432F05140830FF3E031D442F78083A
:100E9000FE39080083169B001C141A088301080001
:100EA000B2242E08F3003008F600F7013108F400F0
:100EB0000319602F6430F6070318F70AF40B5A2F52
:100EC0002F08FD3EF400F41F682F0C30F407831741
:100ED000C4277307F200831F712FF603760A0319E4
:100EE000F703770CF400760CF3006D30F207013055
:100EF000C927F1070318F00AF60B752FF703F71F40
:100F0000752F1F30F2074330C927F1071A30C92760
:100F1000F007F40CF30C3108831F912FB00803196C
:100F2000FF3EF600F302031CF403F60C760C3F3987
:100F300073070318F40AF2077408C927F1070318A6
:100F4000F00A8301F501F3010730FB00F601F70118
:100F50002030F400F30DF20DF10DF00DF60DF70D4C
:100F6000F40D7508F6027B08031C7B0A7702031850
:100F700074147418BE2F7508F6077708F70003106D
:100F8000F40CF40BAA2F080007308A007408F23E14
:100F900082000318013E08008207B734A0343B34B6
:100FA000B934AC349D349F34B034BF34BD34BE3416
:100FB0008F341734AB341F341E349734AE340634B8
:100FC000A13407348A348B343E340A340F34A734C6
:0A0FD000083409343C340B340034BB
:0C0FE40000341F343D345C347A349934FE
:100FF000B834D634F534E23EE23E543EF10A0800FD
:084000000700020004000800A3
:02400E00423F2F
:10420000360020007400750062006500200049003F
:104210004E002D00360020005600460044002000CD
:1042200063006C006F0063006B0020007700690082
:104230007400680020004400430046003700370047
:104240002000730079006E006300680072006F0048
:104250006E002C0020004900320043002000520074
:10426000540043002C002000520047004200200070
:0A4270004C006500640073002E008E
:04427C000800100026
:1042800010001C001800150011001D001900160078
:1042900012001E001A00130017001F001B00000070
:1042A0000F00030009000500300031003400350024
:1042B000320033003F000E000B000A00070006002A
:1042C000030048007000340031004300200020004B
:1042D000560032002E00340038002000320030003A
:1042E000310032002D00300035002D003100320049
:1042F000200044005300310033003000370020001C
:00000001FF
